:100AB5002321323030454655002324323030454617
:020AC5005500DA
:100A7500AF8475840F758A83E4F597F58475C04452
:070A850075CFE4C2C38F84AA
:010A8C002247
:060A04008F27AD27AF268D
:020A0A008D1E3F
:100A0C001209C1EFC454F0F51FAF1E1209C1EF2536
:040A1C001FF51FFFA4
:010A200022B3
:100974008F828E83D3E5829DE5839C501943B70112
:10098400758F03E4F0F58F53B7FE2582F582740466
:060994003583F58380DECF
:01099A00223A
:0206D800A90770
:1006DA0020C3FD20C5FAC2C4D2C5E4FFFC30C3FD65
:1006EA0030C3FDE5C154F8FA64086003BA1011E595
:1006FA001DBF01044401800254FEF5C27C01807CC6
:10070A00BA180B851CC27C02C2C4C2C5806EBA204C
:10071A00028038EA64287030B9010CBC02028015E4
:10072A00EC6404701F8019BC02088BC27C03C2C52A
:10073A008012BC03088DC27C04C2C58007BC0404B5
:10074A00D2C57F01C2C48034BA300AD2C4D2C57CB1
:10075A0009E4FF8027BA3802801EBA4006C2C2C224
:10076A00C58019BA48028010BA50028003BA5808E4
:10077A00D2C47C08AEC28004D2C4D2C5C2C3EC645F
:08078A000860030206EAAF0655
:010792002244
:100AD800AE05AD078E1C8B1DE4FB7F011206D822E4
:100AC700AE03AB05AD078E1C751DA07F021206D8BD
:010AD70022FC
:0603B2008B3D8A3E893FED
:1003B8007547FF75480A7549B57544017545007557
:1003C8004680E4F543F542F541F540E47F50FEFDF3
:1003D800FCAB43AA42A941A840C312066C5031AFF6
:1003E800437BA0E4FD120AD87844E475F0011206B4
:1003F800C8EF12064DAF43AE42AD41AC40E47B01BD
:10040800FAF9F812065F8F438E428D418C4080BB0B
:10041800AB47AA48A949120607FF900080E06F7011
:1004280062900001120620FF900081E06F705490E6
:100438000002120620FF900082E06F7046900003D1
:10044800120620FF900083E06F70389000041206B7
:1004580020FF900084E06F702A900005120620FFAC
:10046800900085E0B5071C900006120620FF90005A
:1004780086E0B5070E900007120620FF900087E07F
:100488006F60037F0022AB3DAA3EA93F120607FF1B
:10049800900091E06F702A900001120620FF9000F2
:1004A80092E0B5071C900002120620FF900093E02E
:1004B800B5070E900003120620FF900094E06F60CD
:1004C800037F0022900089E0F55BA3E0F55DA3E0DF
:1004D800F55E900099E0F557A3E0F559A3E0F55AC9
:0204E8007F0192
:0104EA0022EF
:0D0A21008F0DAF18AE17120A8D8E178F18AB
:020A2E00AC0614
:0D0A3000AB07AF04AD07AF03AB58120AD8F7
:010A3D002296
:0E0AE800E55CC3955B500605580558055C2279
:100A8D000FBF00010ED3EF955EEE955D4006120A85
:050A9D00E8E4FEFF2269
:040277008E088F0955
:10027B00E4F50DF50EF513F514F515F516F517F563
:10028B0018855917855A18855758F50EF50D755C55
:10029B0001E4F512E50D643A6016AF18AE17120AB9
:1002AB002E8F0DAF18AE17120A8D8E178F1880E494
:1002BB000514E51470020513AF18AE17120A2E12AF
:1002CB000A218F0EAD0EAF0D120A0A8F1085101278
:1002DB00120A23120A218F0EAD0EAF0D120A0A75E8
:1002EB0015008F16EF2512F512E516751600F5158C
:1002FB00120A23120A218F0EAD0EAF0D120A0AEF4E
:10030B00421685150A85160BE5162512F512120AEB
:10031B0023120A218F0EAD0EAF0D120A0A8F0FE5B5
:10032B000F2512F512E50F705CF50CE50CC395105B
:10033B005053120A23120A218F0EAD0EAF0D120A63
:10034B000A8F11E5112512F512C3E50B9509E50A84
:10035B009508402DAE0AAF0BBEFB06BFFE0343B1A3
:10036B003043B701758F01850B82850A83E511F048
:10037B00E4F58F53B7FE75B111050BE50B70020554
:10038B000A050C80A6120A23120A218F0EAD0EAF9E
:10039B000D120A0A8F11E5112512700AE50F64017F
:0603AB00600302029C2227
:0103B1002229
:0604EB008B4A8A4B894C8C
:1004F1007554FF75550A7556BE75510175520075D3
:1005010053D0E4F550F54FF54EF54DE47F2BFEFD4C
:10051100FCAB50AA4FA94EA84DC312066C5030AF88
:1005210050E4FBFD120AC77851E475F0011206C8C8
:10053100EF12064DAF50AE4FAD4EAC4DE47B01FA1C
:10054100F9F812065F8F508E4F8D4E8C4D80BCABEB
:1005510054AA55A956120607FF9000D0E06F7062A9
:10056100900001120620FF9000D1E06F70549000BE
:1005710002120620FF9000D2E06F70469000031235
:100581000620FF9000D3E06F70389000041206201F
:10059100FF9000D4E06F702A900005120620FF90B2
:1005A10000D5E0B5071C900006120620FF9000D68A
:1005B100E0B5070E900007120620FF9000D7E06F0C
:1005C10060037F0022AB4AAA4BA94C120607FF9099
:1005D10000DFE06F702A900001120620FF9000E01A
:1005E100E0B5071C900002120620FF9000E1E0B583
:1005F100070E900003120620FF9000E2E06F6003F7
:050601007F00227F01D3
:0106060022D1
:1008B600E48F34F533F532F531AE33AD32AC317801
:1008C600081206958F348E338D328C3178351206A8
:0108D600A879
:0808D7008F678E668D658C644D
:1008DF00AA077808120682A907AF67AE66AD65ACA6
:0F08EF00647810120682AB07AF02AD01120AC780
:0108FE0022D7
:0400A6008E218F22F6
:1000AA00E4F526F527F534F533F532F531F538F56B
:1000BA0037F536F535F53CF53BF53AF53975382B14
:1000CA00F537F536F535F527F526F52CE4F52BE564
:1000DA0026643A60071208D28F2680F3E53C240191
:1000EA00FFE4353BFEE4353AFDE435398F3C8E3B7F
:1000FA008D3AF5391208D28F261208D2120A048FC5
:10010A002985292B1208D28F261208D2120A04E452
:10011A008F30F52FF52EF52DEF252BF52BAE2FADC4
:10012A002EAC2D78081206958F308E2F8D2E8C2DA1
:10013A001208D28F261208D2120A04E5304FFFE5C0
:10014A002FFEE52EFDE52D8F308E2F8D2EF52D8E6F
:10015A00238F24EF252BF52B1208D28F261208D2D3
:10016A00120A048F28E528252BF52BE5286404704C
:10017A00381208D28F261208D2120A041208B68F31
:10018A00261208D2120A04E5344FFFE533FEE5329F
:10019A00FDE5318F348E338D32F531FC781012063D
:1001AA00958F348E338D328C31E528640270381283
:1001BA0008D28F261208D2120A041208B68F261203
:1001CA0008D2120A04E5344FFFE533FEE532FDE5B5
:1001DA00318F348E338D32F531FC78041206958FC7
:1001EA00348E338D328C31E5342524F524E53335CC
:1001FA0023F523E5287058F525E525C39529504FA1
:10020A001208D28F261208D2120A048F2AE52A254A
:10021A002BF52BC3E5249522E5239521402DAE230A
:10022A00AF24BEFB06BFFE0343B13043B701758F4F
:10023A0001852482852383E52AF0E4F58F53B7FEEE
:10024A0075B1110524E52470020523052580AA123B
:10025A0008D28F261208D2120A048F2AE52A252BE1
:0C026A00700AE528640160030200D6223F
:010276002265
:100A3E007F80900000E4F0A3DFFC7B017A00790058
:0C0A4E008B618A6289638A5F8960D2B57F
:010A5A002279
:10093A00AF8475840FE5B0541FFE0560E560AC5FB7
:10094A007002055F14F5828C83EEF0C3E560948033
:10095A00E55F94004006755F00756000C2B5308699
:09096A00FDD2B58F84AF067E00BA
:010973002261
:05000600323732450015
:1009E300E4FBFAC3EB9FEA9E5016900000C3E58236
:1009F3009DE5839C5003A380F40BBB00010A80E3B5
:010A030022D0
:10081500AE8475840F758A83E4F59775840FF58921
:10082500F58475B73075840F4389018D8D758F01FA
:100835008F8EFDFC0DBD00010CE4B505F7ECB40190
:10084500F3438902E58920E4120DEDAA0470010C39
:1008550014D39400EA6480948140E97597028E84EC
:010865002270
:10099B00AF8475840F75E10343E20443E3C075A490
:1009AB000F7580F075A50775AD0775A6FF75A0FFD0
:0509BB0075A7E08F8428
:0109C0002214
:100AA200AF84E4F584759D0443F808759A40D2F842
:020AB2008F842F
:010AB400221F
:03001600020A7566
:1008FF00E4F568F569C2037D207C037FD07E071283
:10090F0009E3120A3EE4F568F56912093AEF641734
:10091F004E7004D20380110569E56970020568C342
:0A092F0094FBE568940940E2A2037E
:01093900229B
:10079300C200C201C20275FFDE75FFAD7D017F0499
:1007A30012081512099B120AA21208FF92003000C8
:1007B3005E1200167BFF7A0079061203B2EF24FF64
:1007C30092013001147D007CDC7F007E40120974AD
:1007D3007F007E4012027780237BFF7A0079061226
:1007E30004EBEF24FF92023002127D007CDC7F00D9
:1007F3007E401209747F007E401200A6E4FFFE0FC4
:10080300BF00010EBE27F8BF10F5E4F584F5C00262
:02081300000ED5
:04000E00024000228A
:01FBFE00FE08
:03000000020A5B96
:03000300025003A5
:03000B000250069A
:030013000250098F
:03001B0002500C84
:0300230002500F79
:03002B000250126E
:0300330002501563
:03003B0002501858
:0300430002501B4D
:03004B0002501E42
:0300530002502137
:03005B000250242C
:0300630002502721
:03006B0002502A16
:0300730002502D0B
:03007B0002503000
:03008300025033F5
:03008B00025036EA
:03009300025039DF
:03009B0002503CD4
:0300A30002503FC9
:100A5B00787FE4F6D8FD9000007F007E20E4F0A3C1
:0A0A6B00DFFCDEFA758169020793D3
:10086600E590540C23C0E0740BC0E0C082C0830244
:100876000B00E590540C23C0E0740BC0E0C082C0AE
:1008860083020B08E590540C23C0E0740BC0E0C053
:1008960082C083020B10E590540C23C0E0740BC099
:0808A600E0C082C083020B18C0
:040B00005390F322F9
:070B080043900C5390F7220B
:070B100043900C5390FB22FF
:040B180043900C22D8
:0708AE00EFC403900B00737F
:10060700BB010689828A83E0225002E722BBFE02F1
:09061700E32289828A83E4932224
:10062000BB010CE58229F582E5833AF583E022508F
:1006300006E92582F8E622BBFE06E92582F8E222D9
:0D064000E58229F582E5833AF583E49322F3
:10064D00BB010689828A83F0225002F722BBFE018C
:02065D00F32286
:0D065F00EF2BFFEE3AFEED39FDEC38FC22EA
:10066C00EB9FF5F0EA9E42F0E99D42F0EC6480C805
:06067C0064809845F022A5
:10068200E8600FECC313FCED13FDEE13FEEF13FF56
:03069200D8F1227A
:10069500E8600FEFC333FFEE33FEED33FDEC33FCC3
:0306A500D8F12267
:1006A8007401FF3395E0FEFDFC080808E6CF2FF63D
:1006B80018E6CE3EF618E6CD3DF618E6CC3CF62216
:1006C800FAE6FB0808E6F925F0F618E6CA3AF62233
:1009C100EF7E0024D0B40A00401624F9B40A004096
:1009D1000CB41000400A24E0B41000400374FFFE80
:0209E100FF22F3
:00000001FF
